:100000000C94A3000C94CB000C94CB000C94CB006C
:100010000C94CB000C94CB000C94CB000C94CB0034
:100020000C94CB000C94CB000C94CB000C94CB0024
:100030000C94CB000C94CB000C94CB000C94CB0014
:100040000C94C4010C94CB000C94CB000C94CB000A
:100050000C94CB000C94CB000C94CB000C94CB00F4
:100060000C94CB000C94CB0007634236B79BD8A707
:100070001A39685618AEBAAB558C1D3CB7CC5763CD
:10008000BD6DEDFD753EF6177231BF000000803F7B
:1000900008000000BE922449123EABAAAA2ABECD97
:1000A000CCCC4C3E00000080BEABAAAAAA3E000009
:1000B0000000BF000000803F000000000008417801
:1000C000D3BB4387D1133D190E3CC3BD4282AD2B38
:1000D0003E68EC8276BED98FE1A93E4C80EFFFBE30
:1000E00001C4FF7F3F00000000000000000023006B
:1000F0002600290000000000240027002A0000003C
:100100000000250028002B00040404040404040457
:1001100002020202020203030303030301020408B2
:100120001020408001020408102001020408102061
:1001300000000008000201000003040700000000A6
:1001400000000000BF0611241FBECFEFD8E0DEBFC5
:10015000CDBF11E0A0E0B1E0ECE3F5E102C0059015
:100160000D92AE30B107D9F721E0AEE0B1E001C0A9
:100170001D92A332B207E1F710E0C3EAD0E004C059
:100180002197FE010E94960AC23AD107C9F70E9440
:100190000E020C949C0A0C940000833081F028F429
:1001A000813099F08230A9F008958730A9F0883025
:1001B000C9F08430B1F4809180008F7D03C08091BC
:1001C00080008F7780938000089584B58F7784BDF9
:1001D000089584B58F7DFBCF8091B0008F77809399
:1001E000B00008958091B0008F7DF9CF1F93CF9319
:1001F000DF93282F30E0F901E05DFE4F8491F90193
:10020000E45EFE4FD491F901E85FFE4FC491CC2328
:10021000A9F0162F81110E94CD00EC2FF0E0EE0F17
:10022000FF1FE250FF4FA591B4918FB7F894EC9166
:10023000111108C0D095DE23DC938FBFDF91CF91E1
:100240001F910895DE2BF8CFCF93DF9390E0FC0150
:10025000E45EFE4F2491885F9E4FFC0184918823C9
:10026000D1F090E0880F991FFC01EC50FF4FA59151
:10027000B491FC01E250FF4FC591D491623071F40A
:100280009FB7F8943C91822F809583238C93E881CB
:100290002E2B28839FBFDF91CF9108958FB7F894BD
:1002A000EC912E2B2C938FBFF6CF1F93CF93DF9320
:1002B000182FEB0161E00E942401209739F460E0DF
:1002C000812FDF91CF911F910C94F600CF3FD10584
:1002D00011F461E0F5CFE12FF0E0E05DFE4FE49135
:1002E000E33031F140F4E130B1F0E230E1F0C03818
:1002F000D1057CF7E4CFE73029F1E83059F1E4305B
:10030000B1F780918000806280938000D0938B0051
:10031000C0938A0004C084B5806884BDC7BDDF91E6
:10032000CF911F91089584B5806284BDC8BDF7CF79
:1003300080918000806880938000D0938900C09372
:100340008800EDCF8091B00080688093B000C093AA
:10035000B300E5CF8091B00080628093B000C0937D
:10036000B400DDCF8E50806480937C0080917A0051
:10037000806480937A0080917A0086FDFCCF809122
:1003800078009091790008951F920F920FB60F9206
:1003900011242F933F938F939F93AF93BF9380919B
:1003A0001F0190912001A0912101B0912201309173
:1003B0001E0123E0230F2D3758F50196A11DB11D15
:1003C00020931E0180931F0190932001A09321018F
:1003D000B093220180911A0190911B01A0911C0100
:1003E000B0911D010196A11DB11D80931A0190933A
:1003F0001B01A0931C01B0931D01BF91AF919F9170
:100400008F913F912F910F900FBE0F901F901895D5
:1004100026E8230F0296A11DB11DD2CFCF93DF9303
:10042000CDB7DEB760970FB6F894DEBF0FBECDBF75
:10043000789484B5826084BD84B5816084BD85B5BF
:10044000826085BD85B5816085BD80916E008160CB
:1004500080936E0010928100809181008260809371
:100460008100809181008160809381008091800073
:100470008160809380008091B10084608093B1009E
:100480008091B00081608093B00080917A00846098
:1004900080937A0080917A00826080937A008091C4
:1004A0007A00816080937A0080917A0080688093DE
:1004B0007A001092C10061E08BE00E94240161E0AB
:1004C00089E00E94240161E083E00E94240162E04F
:1004D00084E00E94240183E28093B00081E0809355
:1004E000B10082E88093800089E1809381008FEFE2
:1004F00090E0909387008093860080E090E0A0E0F9
:10050000BFE38093000190930101A0930201B09397
:1005100003018093040190930501A0930601B09319
:100520000701109208018FEE9EEBADEABEED8093BD
:10053000090190930A01A0930B01B0930C0111E003
:1005400040E0242E40E0342E8FB7F89420911F0114
:100550003091200140912101509122012D873E8749
:100560004F87588B8FBF8EE00E94B201BC01990F5C
:10057000880B990B0E94EF0720E030EC4FE754E422
:100580000E9445072B013C018FE00E94B201BC0193
:10059000990F880B990B0E94EF0720E030EC4FE792
:1005A00054E40E9445074B015C0180E10E94B201C6
:1005B000BC01990F880B990B0E94EF0720E030ECEB
:1005C0004FE754E40E9445076B017C0181E10E94E2
:1005D000B201BC01990F880B990B0E94EF0720E034
:1005E00030EC4FE754E40E94450769837A838B839C
:1005F0009C8383E10E94B201BC01990F880B990B87
:100600000E94EF0720E030EC4FE754E40E944507DA
:100610006D837E838F83988720E030E0A901C3013A
:10062000B2010E94400787FD44C320E030E040E86B
:100630005FE3C301B2010E949F08181634F4412CF5
:10064000512C30E8632E3FE3732EA301920160E04A
:1006500070E088EC92E40E9411092FE632E143E851
:100660005AE30E94A4082B013C0120E030E0A901DC
:10067000C501B4010E94400787FD1FC320E030E0A0
:1006800040E85FE3C501B4010E949F08181634F4E6
:10069000812C912C20E8A22E2FE3B22E2DEC3CECE5
:1006A0004CE45FE3C501B4010E94A4082DEC3CECCE
:1006B0004CEC5EE30E94D30669877A878B879C8720
:1006C00020E030E0A901C701B6010E94400787FD84
:1006D000F8C220E030E040E85FE3C701B6010E94C5
:1006E0009F08181634F4C12CD12C90E8E92E9FE312
:1006F000F92E20E030E0A9016D817E818F819885FF
:100700000E94400787FDE1C220E030E040E85FE35F
:100710006D817E818F8198850E949F08181644F410
:1007200080E090E0A0E8BFE38D839E83AF83B8872D
:100730002D813E814F815885C701B6010E94D406A4
:100740006B017C0120E030E0A9010E94400787FD99
:10075000C1C220E030E040E85FE3C701B6010E947B
:100760009F08181634F4C12CD12C80E8E82E8FE3B2
:10077000F82E20E030E0A90169817A818B819C818B
:100780000E94400787FDAAC220E030E040E85FE316
:1007900069817A818B819C810E949F08181644F49C
:1007A00020E030E040E85FE329833A834B835C83B9
:1007B0002FE832EC45E75CE369817A818B819C818B
:1007C0000E94A4089B01AC016BE37FED8FE79FE3E0
:1007D0000E94D3064B015C0128E431EE4AE75FE357
:1007E0000E94400787FD7FC22BE33FED4FE75FE3A9
:1007F000C501B4010E949F08181644F40BE3802E33
:100800000FED902E0FE7A02E0FE3B02EE4E3F1E002
:100810008491E0E2F1E0F491FD83ECE0F1E0F49109
:10082000F983FF2389F081110E94CD002981E22FF5
:10083000F0E0EE0FFF1FE651FF4FA591B4918C91B0
:100840003D81382381E009F480E010921801109274
:10085000190190911701891771F0809317018D8507
:100860009E85AF85B8898093120190931301A09360
:100870001401B09315018091120190911301A09180
:100880001401B09115012D853E854F855889281B8F
:10089000390B4A0B5B0BDA01C90140910E015091F3
:1008A0000F016091100170911101481759076A07F3
:1008B0007B07B0F49091160180911701981781F091
:1008C00080931601911103C021E0813009F020E0EE
:1008D00020931801913009F4811190E0909319014F
:1008E00080911901882329F0809108018127809344
:1008F00008018091090190910A01A0910B01B0912A
:100900000C01AC01BD013DE0440F551F661F771F70
:100910003A95D1F784279527A627B727AC01BD01C3
:10092000E1E17695679557954795EA95D1F7842744
:100930009527A627B727AC01BD01F5E0440F551F49
:10094000661F771FFA95D1F784279527A627B72723
:100950008093090190930A01A0930B01B0930C01BD
:10096000BD01BB0F880B990B0E94EF0720E030E020
:1009700040E058E30E94A408A70196010E94A40841
:10098000A30192010E94A40820910001309101016D
:1009900040910201509103010E94D406609300012E
:1009A000709301018093020190930301209108014B
:1009B000222371F024EA30E74DE75FE30E94A408A8
:1009C00060930001709301018093020190930301F1
:1009D000C0900001D0900101E0900201F09003016D
:1009E00020E030E0A901C701B6010E94400787FD61
:1009F00083C120E030E040E85FE3C701B6010E9418
:100A00009F08181634F4C12CD12C20E8E22E2FE3D5
:100A1000F22EC0920001D0920101E0920201F09208
:100A2000030120910401309105014091060150918C
:100A30000701C501B4010E94A4082B013C01A501D6
:100A4000940160E070E080E89FE30E94D306A70174
:100A500096010E94A4089B01AC01C301B2010E944F
:100A6000D4064B015C018092040190920501A09292
:100A70000601B0920701A701960169857A858B85E9
:100A80009C850E94D4067B018D83998320E030E011
:100A9000A9010E94400787FD33C120E030E040E813
:100AA0005FE3B7018D8199810E949F0818160CF0B1
:100AB0002CC1B0E0A0E0F0E8EFE320E030E04FE749
:100AC00053E46B2F7A2F8F2F9E2F0E94A4080E9431
:100AD000B70777FD2EC120E030E0A901B7018D8175
:100AE00099810E94400787FD15C120E030E040E871
:100AF0005FE3B7018D8199810E949F0818160CF061
:100B00000EC1B0E0A0E0F0E8EFE320E030E04FE716
:100B100053E46B2F7A2F8F2F9E2F0E94A4080E94E0
:100B2000B7076F3F710511F00CF006C120E030E00F
:100B3000A901B7018D8199810E94400787FDF4C00A
:100B400020E030E040E85FE3B7018D8199810E94A9
:100B50009F08181634F4E12CF12C30E83D834FE364
:100B6000498320E030E04FE753E4B7018D8199815C
:100B70000E94A4080E94B70769837D83A5019401A0
:100B800069857A858B859C850E94D406D62EE72EB2
:100B9000F82E092F20E030E0A9010E94400787FDD0
:100BA000CEC020E030E040E85FE36D2D7E2D8F2D3C
:100BB000902F0E949F0818160CF0C6C0B0E0A0E06D
:100BC000F0E8EFE320E030E04FE753E46B2F7A2FBB
:100BD0008F2F9E2F0E94A4080E94B70777FDC8C0E0
:100BE00020E030E0A9016D2D7E2D8F2D902F0E94E9
:100BF000400787FDAEC020E030E040E85FE36D2DA8
:100C00007E2D8F2D902F0E949F0818160CF0A6C0E5
:100C1000B0E0A0E0F0E8EFE320E030E04FE753E49D
:100C20006B2F7A2F8F2F9E2F0E94A4080E94B70748
:100C30006F3F710511F00CF09EC020E030E0A9017B
:100C40006D2D7E2D8F2D902F0E94400787FD8BC02C
:100C500020E030E040E85FE36D2D7E2D8F2D902F5A
:100C60000E949F0818162CF4D12CE12C90E8F92E44
:100C70000FE320E030E04FE753E46D2D7E2D8F2D04
:100C8000902F0E94A4080E94B7077B0169817D8193
:100C90008BE00E945501B70189E00E9455018981CE
:100CA0008093B4002114310409F44ECC0E9400005A
:100CB0004BCC412C512C3201C8CC812C912C5401AD
:100CC000EDCCC12CD12C760114CD1D821E821F8249
:100CD00018862ECDC12CD12C76014BCD19821A82CB
:100CE0001B821C8265CDB8E48B2EB1EE9B2EBAE739
:100CF000AB2EBFE3BB2E8ACDC12CD12C760189CE81
:100D0000B0E0A0E0F0E0E0E0D8CEBE2DAF2DFD8158
:100D1000E981D3CEB0E0A0E0F0E0E0E0F6CEBE2D79
:100D2000AF2DFD81E981F1CEE12CF12C1D821982DC
:100D300018CF19821D8222CF5FEF5983FBCFB0E01D
:100D4000A0E0F0E0E0E03ECFBD2DAE2DFF2DE02F86
:100D500039CFB0E0A0E0F0E0E0E05ECFBD2DAE2DF9
:100D6000FF2DE02F59CFD12CE12CF12C00E081CFC9
:100D7000F12CE12C8BCFEE24EA94F12C87CFEEE01E
:100D8000F1E082E390E0A0E0B0E080839183A28371
:100D9000B383148215821682178281E0808781874F
:100DA0001286138608955058BB27AA270E94EB0687
:100DB0000C9465080E94570838F00E945E0820F0E5
:100DC00039F49F3F19F426F40C9454080EF4E0957E
:100DD000E7FB0C944E08E92F0E94760858F3BA17E7
:100DE000620773078407950720F079F4A6F50C9441
:100DF00098080EF4E0950B2EBA2FA02D0B01B90127
:100E000090010C01CA01A0011124FF27591B99F080
:100E1000593F50F4503E68F11A16F040A22F232F8C
:100E2000342F4427585FF3CF469537952795A795DC
:100E3000F0405395C9F77EF41F16BA0B620B730B83
:100E4000840BBAF09150A1F0FF0FBB1F661F771FF4
:100E5000881FC2F70EC0BA0F621F731F841F48F4A9
:100E6000879577956795B795F7959E3F08F0B0CF32
:100E70009395880F08F09927EE0F97958795089519
:100E80000E942A0808F481E008950E9459070C94F2
:100E900065080E945E0858F00E94570840F029F447
:100EA0005F3F29F00C944E0851110C9499080C9452
:100EB00054080E94760868F39923B1F3552391F3FF
:100EC000951B550BBB27AA2762177307840738F0B9
:100ED0009F5F5F4F220F331F441FAA1FA9F335D016
:100EE0000E2E3AF0E0E832D091505040E695001CCA
:100EF000CAF72BD0FE2F29D0660F771F881FBB1F84
:100F0000261737074807AB07B0E809F0BB0B802D61
:100F1000BF01FF2793585F4F3AF09E3F510578F08D
:100F20000C944E080C9499085F3FE4F3983ED4F378
:100F3000869577956795B795F7959F5FC9F7880F61
:100F4000911D9695879597F90895E1E0660F771FB3
:100F5000881FBB1F621773078407BA0720F0621B44
:100F6000730B840BBA0BEE1F88F7E09508950E946F
:100F7000BE076894B1110C94990808950E947E08E8
:100F800088F09F5798F0B92F9927B751B0F0E1F04A
:100F9000660F771F881F991F1AF0BA95C9F714C0FA
:100FA000B13091F00E949808B1E008950C9498082F
:100FB000672F782F8827B85F39F0B93FCCF3869533
:100FC00077956795B395D9F73EF490958095709590
:100FD00061957F4F8F4F9F4F0895E89409C097FB0D
:100FE0003EF490958095709561957F4F8F4F9F4F00
:100FF0009923A9F0F92F96E9BB279395F695879544
:1010000077956795B795F111F8CFFAF4BB0F11F406
:1010100060FF1BC06F5F7F4F8F4F9F4F16C08823AD
:1010200011F096E911C0772321F09EE8872F762FE3
:1010300005C0662371F096E8862F70E060E02AF024
:101040009A95660F771F881FDAF7880F9695879510
:1010500097F90895990F0008550FAA0BE0E8FEEFE5
:1010600016161706E807F907C0F012161306E4076C
:10107000F50798F0621B730B840B950B39F40A2665
:1010800061F0232B242B252B21F408950A2609F443
:10109000A140A6958FEF811D811D089597F99F6747
:1010A00080E870E060E008959FEF80EC08950024F0
:1010B0000A941616170618060906089500240A94BD
:1010C00012161306140605060895092E0394000C43
:1010D00011F4882352F0BB0F40F4BF2B11F460FFD2
:1010E00004C06F5F7F4F8F4F9F4F089557FD9058FB
:1010F000440F551F59F05F3F71F04795880F97FBDC
:10110000991F61F09F3F79F0879508951216130695
:101110001406551FF2CF4695F1DF08C016161706C4
:101120001806991FF1CF86957105610508940895F9
:10113000E894BB2766277727CB0197F908950E948B
:101140002A0808F48FEF08950E94B7080C946508E8
:101150000E94570838F00E945E0820F0952311F095
:101160000C944E080C94540811240C9499080E9475
:10117000760870F3959FC1F3950F50E0551F629F5D
:10118000F001729FBB27F00DB11D639FAA27F00DE0
:10119000B11DAA1F649F6627B00DA11D661F829F07
:1011A0002227B00DA11D621F739FB00DA11D621FEC
:1011B000839FA00D611D221F749F3327A00D611D09
:1011C000231F849F600D211D822F762F6A2F1124EB
:1011D0009F5750409AF0F1F088234AF0EE0FFF1F1E
:1011E000BB1F661F771F881F91505040A9F79E3F75
:1011F000510580F00C944E080C9499085F3FE4F37D
:10120000983ED4F3869577956795B795F795E795CA
:101210009F5FC1F7FE2B880F911D9695879597F9D3
:101220000895FA01EE0FFF1F309621053105A1F157
:101230006115710561F48038BFE39B0749F168943B
:101240009038810561F08038BFEF9B0741F099230A
:101250004AF5FF3FE1053105210519F1E8940894AD
:10126000E795D901AA2329F4AB2FBE2FF85FD0F35D
:1012700010C0FF5F70F4A695E0F7F73950F019F051
:10128000FF3A38F49F779F930DD00F9007FC90584A
:10129000089546F00C94540860E070E080E89FE305
:1012A00008954FE79F775F934F933F932F930E944B
:1012B0000C0A2F913F914F915F910E94A4080C94CA
:1012C000690929F416F00C944E080C9498080C94B3
:1012D00054080E947E08A8F39638A0F707F80F92EA
:1012E000E8942BE33AEA48EB5FE70E94BA080F92D2
:1012F0000F920F924DB75EB70F920E94540AE8E624
:10130000F0E00E949B094F915F91EF91FF91E5956D
:10131000EE1FFF1F49F0FE57E0684427EE0F441F01
:10132000FA95E1F74195550B0E94CE090F9007FE03
:101330000C94C2090895DF93CF931F930F93FF92EC
:10134000EF92DF927B018C01689406C0DA2EEF01E8
:101350000E94B708FE01E894A59125913591459129
:101360005591A6F3EF010E94EB06FE019701A8013B
:10137000DA9469F7DF90EF90FF900F911F91CF9172
:10138000DF9108959B01AC0160E070E080E89FE38D
:101390000C9445070C944E080C94880A0E947E0811
:1013A000D8F39923C9F3940F511DA3F391505040E2
:1013B00094F059F0882332F0660F771F881F915000
:1013C0005040C1F79E3F51052CF7880F911D96950F
:1013D000879597F908955F3FACF0983E9CF0BB2746
:1013E000869577956795B79508F4B1609395C1F7A1
:1013F000BB0F58F711F460FFE8CF6F5F7F4F8F4F3F
:101400009F4FE3CF0C94990816F00C94880A0C9423
:10141000540868940C944E080E947E08A8F39923FF
:10142000C1F3AEF3DF93CF931F930F93FF92C92FB6
:10143000DD2788232AF02197660F771F881FDAF7A8
:1014400020E030E040E85FEB9FE3883920F0803E09
:1014500038F021968F770E94D406E0E9F0E004C0CE
:101460000E94D406EDEBF0E00E949B098B01BE01C7
:10147000EC01FB2E6F5771097595771F880B990B3F
:101480000E94EF0728E132E741E35FE30E94B708DB
:10149000AF2D9801AE01FF900F911F91CF91DF9179
:1014A0000E94EB060C946508FA01DC01AA0FBB1F31
:1014B0009B01AC01BF5728F42227332744275078DB
:1014C00020C0B75190F4AB2F00244695379527954F
:1014D000011CA395D2F3002071F0220F331F441F8B
:1014E000B395DAF30ED00C94D30661307105A0E801
:1014F0008A07B94630F49B01AC0166277727882715
:101500009078309621F0208331834283538308956D
:101510009F3F31F0915020F4879577956795B79567
:10152000880F911D9695879597F90895EE0FFF1FE7
:0C1530000590F491E02D0994F894FFCF91
:0E153C000000003F0000003F00EFBEADDE00EB
:00000001FF
